:0300000002000EED
:03000300020028D0
:20000B0002001F75810DD2AFD2A912002B80FE12001B80FB758CDC758A00050832050832F8
:20002B007400F50D7411F50C743BF50B7400F50A748075F025C0E0C0F012029315811581F6
:20004B00E50812031D7B0A12031412036A45F0700302006202004B7400F5081200701200EB
:20006B00F102004B22E50904F50914E50975F0007B0A7C001203B645F070030200F07400E4
:20008B00F509E50D4401F50DE50A04F50A14E50A75F0007B3C7C001203B645F0700302001C
:2000AB00F07400F50AE50D4402F50DE50B04F50B14E50B75F0007B3C7C001203B645F07098
:2000CB00030200F07400F50BE50C04F50C14E50C75F0007B187C001203B645F070030200C8
:2000EB00F07400F50C22E50D540175F0007B007C0012039345F0700302013D74F275F0036D
:20010B00C0E0C0F0E50C75F000C0E0C0F0E50B75F000C0E0C0F0E50A75F000C0E0C0F07421
:20012B000475F00012013E7FF81202FEE50D54FEF50D2223F42581F8868208868308E4FE51
:20014B00FF93700122B42555A3E493B42D06430780A3E493B4300343074024D0B40A0050E9
:20016B000CCE75F00AA42EFEA3E49380EDE493B46413E60886F030F708430720120360A61A
:20018B00F018F68003B4750543070A801CB478054307108014B46F0B430708800C1202D0A6
:2001AB00A3809BB462624307027A00C004C005C006C007AB0753031F7C00E60886F0120306
:2001CB0026A6F018F6EDD007D006D005D0042430B43A0040022407C0E00AE645F070CCA9AE
:2001EB0002EF30E506742D1202D00A120274D0E01202D0D9F90808EF30E7A5EAC39E50A075
:20020B0074201202D00A80F3B4630BAA01120274E61202D080DFB4732BC082C08386820879
:20022B0086837A00E4936004A30A80F88683188682120274E493A360051202D080F6D08353
:20024B00D08280B1B4691986017A00E76004090A80F91202748601E7609B1202D00980F7AD
:20026B00F97A01120274E980A8EE601B8FF020F716C002EAC39E500D742030F60274301275
:20028B0002D00A80EED0022278FB1202F28603088604748075F070120326120360758921E9
:2002AB00F58DF58B7588597598522278FB1202F28682088683E493602D1202D0A380F6784F
:2002CB00FB1202F2E63099FDC299F599B40A17740D80F2E430980C3098FDC298E599B40D9F
:2002EB0002740A75F00022C82581C822C92581C97A0022D083D082CF2581F581CFC082C05F
:20030B008322CF2581F581CF227C00CB30E7011CCB2275F00030E70215F022C002C001AA17
:20032B00F0F97E007D007F11C3E933F9EA33FADF08F5F0E9D001D00222ED33FDEE33FEC3D6
:20034B00ED9BF5F0EE9C40E0ADF0FED380DB14B4FF0215F022120359F4C5F0F4C5F02212CE
:20036B0003BD4029801E1203BD40227017801E1203BD40107017800C1203BD501080051254
:20038B0003D16009E4F5F0221203D160F7E4F5F004221203D140F680EB1203D140EF70E40E
:2003AB0080EB1203D140DD70E480D91203D150DD80D2C39BC5F09C20E70720D207C345F004
:2003CB002220D2F9D322C5F0C39C7003E5F09B22FBE493CB22FCE493FB740193CC22FAE456
:1803EB0093F9740193CA220A20253032753A253032753A2530327500E8
:00000001FF
